:04100000A0EF3FF02E
:107F40000001BEEF3FF008D0100E056E940EE82E33
:107F5000FED7052EFCD700D0FF0E0126FF0E022211
:107F6000FF0E0322FF0E04220128EEE10228ECE1BD
:107F70000328EAE10428D8B41200E6D7000E946E74
:107F8000000E826E000E956E000E836ECB68070E9B
:107F9000CA6E3C0EBD6E3C0EBA6E000E066E7F0EB3
:107FA000066401D014D006C08CFF06C0BEFF065088
:107FB0000008800FBB6E640E016E000E026E000E94
:107FC000036E000E046EA3EC3FF0062AE8D77F0E86
:107FD000066E0650D8B4E1D706C08CFF06C0BEFFBF
:107FE00006500008800FBB6E640E016E000E026E1C
:107FF000000E036E000E046EA3EC3FF00606E9D7F8
:020000040020DA
:08000000FFFFFFFFFFFFFFFF00
:020000040030CA
:0E000000240E3F1EFF8181FF0FC00FE00F4056
:00000001FF
